:1074000080E189BD82E189BD09B400FEFDCF089508
:10741000D3D569F08091E9008F931092E900A5D44B
:1074200083FF01C027D58F9187708093E90008956D
:107430008EEF0090E10008220092E1000895F20131
:10744000F999FECFF2BDE1BD0895F9DFF89A80B554
:1074500008C0F5DF1FBA80BD0FB6F894FA9AF99A02
:107460000FBE31962F010895E0E0F0E085919491F0
:107470000196089580EE8BB98BEA37D0109289007F
:107480008AEF8093880082E080936F0083E080938E
:1074900081004AD049D05C98EDE6F7E785913AD073
:1074A000E038E1F781E08093D7008AE482BF109250
:1074B000D8001092E2001092DA001092E10080E809
:1074C00008D019BC1EBA1092E00065D489E056D4E9
:1074D00081E98093D8000895A3E6B1E090E81AD03E
:1074E0008D939A95E1F7089586E008D010C083E067
:1074F00005D08F2F0FD08E2F0DD080E05E9A599837
:1075000009C005D085E0FADF05D080FDFDCF599A8E
:107510005E9808958EBD8DB587FFFDCF8EB5089519
:107520008FE08221E9F7F3DFE3E6F6E05C9A40E4DE
:1075300058E06081718198E08FEF60FF8F7070FF7D
:10754000807FE8DF669576959A95B1F7E058FF4F12
:107550005A9579F7EE5FF3404A9551F70895E3E6BF
:10756000F1E097FC38C094FC4FC092FE08958684E9
:10757000882011F4992459C0F894C089D78520E057
:1075800030E080E090E4AFEFBFEF119688199040B3
:10759000E0F72D01BD4F8D0127FD13C0E0E0F8E0BD
:1075A00011928EE7819392E4E11791939AE508F0A6
:1075B00092E4E334C9F781931082B5DFFE0121968E
:1075C00096DF8ADFF901FBD420583F4F040D151DCB
:1075D0008A9411F71EC28301282D60906C0170906F
:1075E0006B0141D019F48823C1F70895380188242C
:1075F0003AD0B9F580916A01821709F4830160904D
:107600006E0170906D01F4CF60906E0170906D010D
:107610002AD059F48823C1F708959FEF95FC03C041
:1076200096FE089591E097FB890E662477248301E6
:10763000222719D0B1F48823A1F380916A0136F092
:10764000881650F4821730F0213003C0881520F4DA
:10765000281710F48301282F60906E0170906D013F
:10766000E8CF3801822EF30142DF36DFC3E6D1E0F6
:10767000E6E6F7E709908591081621F4ED36D1F793
:107680000880801044CFC9E029DFCA95E9F7D0E12E
:1076900095FC1EC097FC53C094FC35C0C3E6D2E0F5
:1076A000E3E6F6E098E088E78E0F00840192E817A1
:1076B000E1F7884F09900192E817E1F7C858DF4FCA
:1076C0009A9589F72DDFC85FD340C33E49F749C07B
:1076D000C3E6D6E0EBE5FAE098E08E2F88570290FB
:1076E0000086E817E1F738960A900292E817E1F76A
:1076F0003897C857D0409A9581F712DFC850DC4FB1
:10770000C33E41F72EC0A3EEB6E0E3E6F6E09AE012
:10771000C6E00D9080818025807F802582958193B1
:10772000A336B90709F4B2E0E336F90709F4F2E049
:10773000E336FC0771F7F4DEDA9529F712C0A3EE01
:10774000B9E0E3E6FAE092E00E90829180258F7036
:10775000802582958083E336F907B1F7E1DEDA957B
:1077600071F78827089541524455424F5915003FFB
:1077700075104FA055A100A200A87F81CFB121AF05
:107780000000FFFFCFCFFFFFFFFFCFCFFFFF0000C5
:10779000FE067E7E06FE46565616FE0656461EFE21
:1077A0003F61E9E3FFE3EBE3FFE3EBE3FFE16B3F83
:1077B00012011001020000084123370001000000FF
:1077C000000109023E0002010080320904000001AC
:1077D000020201000524001001042402040524060D
:1077E0000001070582030800FF09040100020A00E6
:1077F00000000705040210000107058302100001C4
:1078000011241FBE04B714BE88E18093600010925B
:1078100060008EEF9AE09EBF8DBF222433242101A9
:107820004394310141018AC00F928F939F931F921D
:107830000FB60F9211244F936F938091DA0080FF5F
:1078400037C023C00F920FB68F939F93EF93FF9390
:1078500088278093850080938400E0E5F1E09281A1
:10786000907261F490818917980B908309F45D9868
:1078700091818917980B918309F42898239411F426
:107880008315381EFF91EF9154C08091D80080FF7E
:107890000FC08091DA008E7F8093DA008091D9004A
:1078A00080FF04C0ADDD81E08EBB02C019BC1EBAF2
:1078B0008091E10080FF0BC05BD280FF08C05BD2EB
:1078C0008091D800806205DE19BC85E08EBB809176
:1078D000E10084FF1AC04CD284FF17C091DD809173
:1078E000D8008F7DF6DD8FEEA4DD42D28F7E8160E1
:1078F00045D280915301882331F48091E30087FDC4
:1079000002C081E001C084E08EBB8091E10083FF72
:107910000CC02ED283FF09C087EF8BDD82E08EBBC7
:107920001092530185DD27D236D26F914F910F907F
:107930001F909F918F910FBE0F90189580E88093B4
:10794000610010926100B1E0B5BF82E085BF80EFB9
:1079500085B987EE84B91DB8769A10BA80EF81BBDD
:1079600082E68BB982EF8AB980E58CBDBDBDA0E00F
:10797000E0EBF7E705900D92A035E1F78C911D92B1
:10798000BB30E1F701FF10C08B3A71F45F9A89EBCD
:10799000ACDD80E880BF8DEA8093640089E9809344
:1079A000650085E083BF889500FF07C07C9B05C00C
:1079B0004CDD882312F058DD61F55CDD789453DEF0
:1079C00071F0ABE9B7E0E0E8F7E790E105900D92E0
:1079D0009A95E1F7A059BF4FE03BB9F7A5DD56D026
:1079E00017DD80915201807881F48FB18095807F7E
:1079F00066991C9B8460982E10DE8BEA8825809304
:107A0000FF0A8110ACDD92FC02C0332042F72CDD6E
:107A100031F3F89489EB69DD81E08093E000109206
:107A20006F0010928100109285001092840081E016
:107A300085BF15BE2E9A2F9A2D9A5D9828980C9482
:107A4000000091D107C053D102C0B6D239F08DD118
:107A500082FFFBCF85FFF7CF8091F1000895082EBC
:107A600083E082D185FD07C077D102C0A5D269F03D
:107A70007CD180FFFBCF0092F10080915201807297
:107A800021F45D9A84E68093500108956CD182FFC1
:107A900034C180915201807221F4289A84E6809347
:107AA0005101CFDF182F853431F422248EE7382E90
:107AB000C6DC8DE007C1843511F4C3DFFACF8C3406
:107AC000C1F38035B1F3843721F484E4C8DF80E06A
:107AD000F9C0813611F489E5F5C0813429F4B1DFAC
:107AE000582EAFDF482EE5CF803711F483E5EAC08A
:107AF000833539F4E6E6F7E78591B1DFED36E1F756
:107B0000E2C0863521F481E3AADF86E3DBC0863755
:107B100061F481E3669B8E5F1C9B8F5FA0DF8FB15A
:107B2000809582958F708F5BCDC08837A9F489DFEF
:107B300080935201289884FD289A5D9883FD5D9A70
:107B40002E9A81FD2E982F9A82FD2F982D9A80FDD6
:107B50002D9887FD8824ADCF8A3649F48FE9CEDC95
:107B6000C3E0D8DC7CDFCA95E1F7D1DCACC0833759
:107B700031F487E874DF85E972DF8EE1A3C08536D2
:107B800039F4E0E8F3E72ED2E058F040E0F791CF87
:107B9000823631F489E563DF80E061DF80E892C0FE
:107BA000823419F0873609F079C033244ADFD82FA0
:107BB00048DFC82F46DF082F8354843008F081C087
:107BC000063411F4440C551CF20110926F00173664
:107BD000A1F4033471F483E08BDC9CDC40DF21975B
:107BE000E1F795DC08C0063411F4859101C02DDC65
:107BF00036DF2197C2F72F0149C00334A1F48E2F3D
:107C0000882321F471DC88ED73DC7BDC6DDC82E0A1
:107C10006FDC17DF7FDCCA95E1F773DC3196DA950C
:107C200071F72F0131C00634F1F49F01F437D8F415
:107C3000D9D119C006DF063461F4C0FB46F0F43731
:107C400028F4182E81E087BFE89511243296082E7B
:107C50000AC0043439F4DF01B370AD59B94F8D93C4
:107C6000319601C0F6DB21972AF7043431F42F0155
:107C7000F370FE2B49F458DC07C0063429F42F01B9
:107C8000F901F43708F4ACD18DE0E9DE063411F4E3
:107C90005694479482E080936F0015C08237E1E0EC
:107CA00049F08634E0E031F08E34E3E019F08135BC
:107CB00031F4E2E0F0E089E087BF849103C08B31CA
:107CC00011F08FE3CCDE83E0B0DB46D095FF03C03C
:107CD00009C072D191F049D080FFFBCF3DD002C0E6
:107CE0006BD159F042D080FFFBCF84E09EDB8BE765
:107CF00034C060D1E4E5F1E067E0089590915B0164
:107D000080915C01913231F0913A61F5813251F507
:107D1000F0DF72C0803231F5ECDF4ED1E9F0853012
:107D2000D9F023D083FD18C082FFF7CF04C094DEC2
:107D30008193615031F09091F3008091F200892B92
:107D4000B1F7D5DF611549F704C036D129F0853088
:107D500019F00BD080FFF9CF8EE79091E8008923CE
:107D60008093E800089584E060DB8091E800089546
:107D70008091E2000895FCDF8E7F80618093E200B5
:107D8000089582E061EC09D083E061E802D084E0EC
:107D900060E842E103C080E060E042E046DB81E071
:107DA00007D01092ED006093EC004093ED00089531
:107DB0009091EB00892B8093EB00089560E0923066
:107DC00029F0913031F4E0E062E103C0E2E16EE3DA
:107DD00000C0F1E0089580915B0188234CF402C05B
:107DE000EBD0C1F3C2DF82FFFBCF81CFE5D091F3AF
:107DF000BCDF80FFFBCFB0CF4091610150916201A9
:107E00004617510510F490E028C0611511F0462F77
:107E1000FACFA2DF40E0F7CFCFD059F1853049F15A
:107E2000A4DF83FD64CFA1DF82FD20C080FF15C0E9
:107E30003091F3002091F20005C081918093F10010
:107E400041502F5F411519F028303105B0F350E053
:107E50002830310509F451E07FDF4115E9F655235B
:107E6000D9F604C0A9D029F0853019F07EDF82FF51
:107E7000F9CF3DCFEBE5F1E0EFDD8193E336E1F7BC
:107E80003DDF73DF83FF91C080915B0190915C01C6
:107E9000913009F170F09330F1F0953009F444C05D
:107EA000963009F456C0983009F460C0993059F7FB
:107EB00067C0823841F780915F01B6DA2091EB000C
:107EC0001092E90077D02295269521702093F10039
:107ED0001092F10052C0882311F08230A1F68F7108
:107EE000823089F680915D018823D1F420915F0171
:107EF000277049F22093E9008091EB0080FF10C0C9
:107F0000933011F480E20BC080E152DF81E0880FF2
:107F10002A95E9F78093EA001092EA0088E048DFAA
:107F20001092E90047D02AC0882391F410915D0196
:107F300010680FB7F8943ED04EDF17DF80FFFDCFFB
:107F40001093E300103883E009F482E08EBB0FBF8A
:107F50002CC08058823048F580915D0190915E017F
:107F60002DDF603011F126D047DF1FC08038E9F4E3
:107F700021D0809153018093F100EEDE2CDF15C0FB
:107F8000882399F490915D01923078F49093530195
:107F900011D021DF80915301882321F48091E300E7
:107FA00091E087FD94E09EBBECDEDFDE83FF089569
:107FB00080E2FEDE87EFD1CE8EB388230895A3E65C
:107FC000B1E0F437B8F40ED090E40D901D9081E04C
:107FD00087BFE89532969A95C1F71124E058F04092
:107FE00085E001C083E001D081E187BFE89507B655
:067FF00000FCFDCF089526
:047FFC00E2CFFBDCF9
:040000030000740085
:00000001FF
